:040000008031202803
:100008007E14803120007F08F2002100931C132801
:100018002000931C13288231B62280311B2821002E
:10002800911C1B282000911C1B288231C9227208B0
:100038002000FF007E10090080312228F901FA0112
:1000480020308400003085004030833121237E1029
:1000580020008131F7292000E300E1018231FA22F2
:100068008031F40074082000E100E11F32286108A3
:100078007F39F400630886008701740881008231A3
:10008800FA228031F4002000630A86008701740890
:1000980081006308860087010108FD3EF4006308BB
:1000A8000A3E8600870174088100E201630A86001F
:1000B800870163088400850100080107F4007408BB
:1000C800E000E20163080A3E860087010108620237
:1000D80003188C288231FA228031F400200062084B
:1000E800023E6307F50075088600870174088100E1
:1000F8006208023E6307F40074088600870101085D
:10010800F5007508E0070130F4007408E207662876
:1001180063080B3E860087010108F40063080C3E63
:1001280086008701740881006308023E8600870103
:100138000108F40063080B3E8600870174088100FB
:100148006308033E860087010108F40063080D3E3A
:1001580086008701740881008231FA228031F40018
:10016800200063080E3E86008701740881000D3068
:10017800F500FB30F400F40BBF28F50BBF28003264
:10018800200063080E3E860087017F306005F4007A
:10019800740801060319D22801300800003008004D
:1001A8002000E500650886008701413FA500650835
:1001B800860087014D3FCF0065080B3E860087010A
:1001C80002300106031DF128A601A7010230E40050
:1001D8006408CE008D158D143C2965080B3E8600F9
:1001E800870104300106031D062965080C3E8600B8
:1001F800870102300106031D06297030E4006408F7
:10020800A600232965080B3E8600870104300106F5
:1002180003192C293C291A30E4006408CE00033065
:10022800E4006408A3003A29173025290A30230678
:10023800031D2029A301A30A1D302529A601A70112
:100248000230E4006408CE003A29A601A7013A2941
:100258004F08013A03191A29033A03191829013AD0
:1002680003190F290C3A0319222929298D158D10F4
:100278004E08043EE4006408A40023308131C621FE
:1002880080312000E4006408D000233081317121DE
:100298008031033020002306031D62290F304F06EA
:1002A800031D62290A30E4006408A3000330E40057
:1002B8006408A6002330813171210800200023033F
:1002C800031D08000F304F06031D0800A301A601F7
:1002D800A60A23308131712108002000E300033091
:1002E800E1009730E000E00B7729E10B7729003235
:1002F8002000E201630A8600870101088038823104
:10030800A222813120006308023E8600870101088D
:100318008231A2228131200063082C3E86008701A9
:1003280001088231A22281312000E20163082B3EBC
:1003380086008701010862020318B3296208033E98
:100348006307E00060088600870101088231A22265
:10035800813101302000E0006008E2079A29630833
:100368002D3E8600870101088231A22281310630A4
:100378002000E1003030E000E00BC029E10BC0298B
:1003880000000800F70077082C3E860087017708F0
:10039800023E840085010008F300770A8400850185
:1003A800000873070107F4007408F500F601F60168
:1003B80077082B3E86008701010876020318F42986
:1003C8007608033E7707F300730886008701010863
:1003D800F4007408F5070130F3007308F607DC2908
:1003E80075087F3908008231EB2281318B170B1792
:1003F8002000E7018D14042A51308031D420813146
:10040800823161228131513080312F2081312000A9
:10041800E6006608E80083313F2381312000680840
:100428000319002A01302000E6006608A2070530FB
:100438002202031C242A23001D121D162000A201DB
:100448008D148D11042AF5007508F3007308F60061
:100458007636F3007308F6067608F3000230F336B2
:10046800890B332A7308F4007408F6067608F3003B
:100478000430F336890B3D2A7308F4007408F60635
:1004880076080139080022008D018C011C302300F8
:100498008C0010308D00203024008C00F5308D0049
:1004A800F53021008D00FF308C0095178030220038
:1004B8009D0001309E008B1108007B3028009700BA
:1004C80026309600950120009310210093144E3099
:1004D800F3000330F4008331272382312000A00188
:1004E800A1018331422308007B3020009C00263084
:1004F8009B009A019110210091144F30F3000330B2
:10050800F40083312D238231F901FA018331452327
:1005180008007B3020009C0026309B009A01911037
:10052800210091144F30F0000330F100833139235A
:100538008231F901FA01833148230800F8002000CC
:10054800111EA32A7808823127228231F700770CFE
:10055800031CB12A23001E14B32A23001E10780896
:100568009A000800200093100130A0070030A13D38
:1005780000302102C83003192002031C0800823110
:10058800DB222000A001A101080020009110013009
:10059800F9070030FA3D00307A0232300319790247
:1005A800031C080083310823F901FA010800200020
:1005B8006B086C04031908006C088A006B080A00B1
:1005C800823182318D22823183314B23080082317E
:1005D8004722823183313323823182316122823151
:1005E8008231782282318331162308002000911E3F
:1005F800FA2A23009D1C022B1D121D1600301D18FF
:100608000130F30019080800200069086A0403197A
:10061800080002308D068D116A088A0069080A00F0
:1006280083310800083023009F00D0309D006430DB
:100638009E00CF309B009C010800640080010131BE
:10064800890B222B003474082000EC007308EB009F
:10065800080074082000EA007308E90008007030F8
:10066800210099009A019801080071082000EA0009
:100678007008E900080020001C1108002800171560
:10068800080020001C15080020001C150800280080
:0806980017110800080008001A
:020000040001F9
:04000E00E4F9FFDE34
:00000001FF
